:1000000000308A001928000010308400000803190D
:10001000182801308D008C018C0B0C288D0B0B28BF
:100020004A308C008C0B122800000000800B09283D
:10003000402884011F3083058316811708308312FE
:100040008C008C1D2B280730810181308400000832
:10005000C0390F3880006400813084000008C03946
:100060000C048000831606148312061C4328831692
:1000700085118312851502308F00FA309000042814
:100080008F0B3D284728831685118312851132284E
:0200900063000B
:02400E00FE3F73
:00000001FF
